 pcie950_ser

 Timestamp is 474fcaf0 (Fri Nov 30 08:33:52 2007)

 Preferred load address is 10000000

 Start         Length     Name                   Class
 0001:00000000 0000029cH .rdata                  CODE
 0001:0000029c 00000064H .rdata$debug            CODE
 0001:00000300 000066bcH .text                   CODE
 0001:000069bc 00000244H .xdata                  CODE
 0001:00006c00 00000028H .idata$2                CODE
 0001:00006c28 00000014H .idata$3                CODE
 0001:00006c3c 000000d8H .idata$4                CODE
 0001:00006d14 000000acH .idata$6                CODE
 0001:00006dc0 00000107H .edata                  CODE
 0002:00000000 000000d8H .idata$5                DATA
 0002:000000d8 00000004H .CRT$XCA                DATA
 0002:000000dc 00000004H .CRT$XCZ                DATA
 0002:000000e0 00000004H .CRT$XIA                DATA
 0002:000000e4 00000004H .CRT$XIZ                DATA
 0002:000000e8 00000004H .CRT$XPA                DATA
 0002:000000ec 00000004H .CRT$XPZ                DATA
 0002:000000f0 00000004H .CRT$XTA                DATA
 0002:000000f4 00000004H .CRT$XTZ                DATA
 0002:000000f8 00000004H .data                   DATA
 0002:000000fc 00000014H .bss                    DATA
 0003:00000000 000003f0H .pdata                  DATA

  Address         Publics by Value              Rva+Base     Lib:Object

 0001:0000001c       ??_C@_1BI@LAHN@?$AAP?$AAr?$AAi?$AAo?$AAr?$AAi?$AAt?$AAy?$AA2?$AA5?$AA6?$AA?$AA@ 1000101c     mdd.obj
 0001:00000034       ??_C@_1CC@CKAL@?$AAD?$AAe?$AAv?$AAi?$AAc?$AAe?$AAA?$AAr?$AAr?$AAa?$AAy?$AAI?$AAn?$AAd?$AAe?$AAx?$AA?$AA@ 10001034     mdd.obj
 0001:00000058       ??_C@_1CE@GCBE@?$AAF?$AAl?$AAo?$AAw?$AAC?$AAt?$AAr?$AAl?$AAH?$AAi?$AAg?$AAh?$AAL?$AAe?$AAv?$AAe?$AAl?$AA?$AA@ 10001058     ser16950.obj
 0001:0000007c       ??_C@_1CC@MJNM@?$AAF?$AAl?$AAo?$AAw?$AAC?$AAt?$AAr?$AAl?$AAL?$AAo?$AAw?$AAL?$AAe?$AAv?$AAe?$AAl?$AA?$AA@ 1000107c     ser16950.obj
 0001:000000a0       ??_C@_1BO@HEHB@?$AAR?$AAx?$AAI?$AAn?$AAt?$AAT?$AAr?$AAi?$AAg?$AAL?$AAe?$AAv?$AAe?$AAl?$AA?$AA@ 100010a0     ser16950.obj
 0001:000000c0       ??_C@_1BO@EEEJ@?$AAT?$AAx?$AAI?$AAn?$AAt?$AAT?$AAr?$AAi?$AAg?$AAL?$AAe?$AAv?$AAe?$AAl?$AA?$AA@ 100010c0     ser16950.obj
 0001:000000e0       ??_C@_1CE@MAOK@?$AAB?$AAa?$AAu?$AAd?$AAr?$AAa?$AAt?$AAe?$AAM?$AAa?$AAp?$AAL?$AAi?$AAs?$AAt?$AAT?$AAo?$AA?$AA@ 100010e0     ser16950.obj
 0001:00000104       ??_C@_1CI@IFEI@?$AAB?$AAa?$AAu?$AAd?$AAr?$AAa?$AAt?$AAe?$AAM?$AAa?$AAp?$AAL?$AAi?$AAs?$AAt?$AAF?$AAr?$AAo?$AAm?$AA?$AA@ 10001104     ser16950.obj
 0001:0000012c       ??_C@_1CC@JFGI@?$AAC?$AAr?$AAy?$AAs?$AAt?$AAa?$AAl?$AAF?$AAr?$AAe?$AAq?$AAu?$AAe?$AAn?$AAc?$AAy?$AA?$AA@ 1000112c     ser16950.obj
 0001:00000210       IoVTbl                     10001210     oxser.obj
 0001:00000288       ??_C@_1BE@MJOB@?$AAR?$AAe?$AAg?$AAS?$AAt?$AAr?$AAi?$AAd?$AAe?$AA?$AA@ 10001288     oxser.obj
 0001:00000300       DoTxData                   10001300 f   mdd.obj
 0001:0000047c       DoRxData                   1000147c f   mdd.obj
 0001:00000554       RxBytesAvail               10001554 f i mdd.obj
 0001:00000574       SerialEventHandler         10001574 f   mdd.obj
 0001:0000067c       StartDispatchThread        1000167c f   mdd.obj
 0001:00000794       StopDispatchThread         10001794 f   mdd.obj
 0001:00000828       ApplyDCB                   10001828 f   mdd.obj
 0001:00000924       COM_Init                   10001924 f   mdd.obj
 0001:00000bb4       COM_Open                   10001bb4 f   mdd.obj
 0001:00000e34       COM_Close                  10001e34 f   mdd.obj
 0001:00000fa4       ProcessExiting             10001fa4 f   mdd.obj
 0001:000010b8       COM_Deinit                 100020b8 f   mdd.obj
 0001:000011b8       COM_Read                   100021b8 f   mdd.obj
 0001:00001460       COM_Write                  10002460 f   mdd.obj
 0001:000015d4       COM_Seek                   100025d4 f   mdd.obj
 0001:000015dc       COM_PowerUp                100025dc f   mdd.obj
 0001:00001600       COM_PowerDown              10002600 f   mdd.obj
 0001:00001638       WaitCommEvent              10002638 f   mdd.obj
 0001:00001750       EvaluateEventFlag          10002750 f   mdd.obj
 0001:000017f0       COM_IOControl              100027f0 f   mdd.obj
 0001:000021bc       OxserGetBaudConfigFromBaudRate 100031bc f   ser16950.obj
 0001:0000233c       ReadPortChar               1000333c f   ser16950.obj
 0001:0000234c       ReadRegisterChar           1000334c f   ser16950.obj
 0001:0000235c       WritePortChar              1000335c f   ser16950.obj
 0001:0000236c       WriteRegisterChar          1000336c f   ser16950.obj
 0001:00002384       ClearPendingInts           10003384 f   ser16950.obj
 0001:00002444       ReadLSR                    10003444 f i ser16950.obj
 0001:000024a8       ProcessLSR                 100034a8 f i ser16950.obj
 0001:0000252c       ReadMSR                    1000352c f i ser16950.obj
 0001:00002594       ProcessMSR                 10003594 f i ser16950.obj
 0001:000025e0       InstallSoftwareISR         100035e0 f   ser16950.obj
 0001:0000284c       SL_Open                    1000384c f   ser16950.obj
 0001:00002b08       OUTB_650_REG               10003b08 f i ser16950.obj
 0001:00002bc0       OUTB_ICR_REG               10003bc0 f i ser16950.obj
 0001:00002c4c       SL_Close                   10003c4c f   ser16950.obj
 0001:00002cf0       SL_Init                    10003cf0 f   ser16950.obj
 0001:00002e58       SL_PostInit                10003e58 f   ser16950.obj
 0001:00002e74       SL_ClearDTR                10003e74 f   ser16950.obj
 0001:00002efc       SL_SetDTR                  10003efc f   ser16950.obj
 0001:00002f84       SL_ClearRTS                10003f84 f   ser16950.obj
 0001:0000300c       SL_SetRTS                  1000400c f   ser16950.obj
 0001:00003094       SL_ClearBreak              10004094 f   ser16950.obj
 0001:0000311c       SL_SetBreak                1000411c f   ser16950.obj
 0001:0000319c       SetBaudRate                1000419c f   ser16950.obj
 0001:00003238       WRITE_DIVISOR_REG          10004238 f i ser16950.obj
 0001:00003314       SL_SetBaudRate             10004314 f   ser16950.obj
 0001:000033bc       SL_SetByteSize             100043bc f   ser16950.obj
 0001:000034ac       SL_SetParity               100044ac f   ser16950.obj
 0001:000035b0       SL_SetStopBits             100045b0 f   ser16950.obj
 0001:0000366c       SL_GetRxBufferSize         1000466c f   ser16950.obj
 0001:00003674       SL_GetInterruptType        10004674 f   ser16950.obj
 0001:00003834       ReadASR                    10004834 f i ser16950.obj
 0001:00003918       SL_RxIntr                  10004918 f   ser16950.obj
 0001:00003d28       BytesInFifo                10004d28 f i ser16950.obj
 0001:00003e1c       SL_TxIntrEx                10004e1c f   ser16950.obj
 0001:00004190       SL_LineIntr                10005190 f   ser16950.obj
 0001:0000421c       SL_OtherIntr               1000521c f   ser16950.obj
 0001:00004328       SL_ModemIntr               10005328 f   ser16950.obj
 0001:00004340       SL_GetStatus               10005340 f   ser16950.obj
 0001:000044b0       INB_650_REG                100054b0 f i ser16950.obj
 0001:00004570       SL_Reset                   10005570 f   ser16950.obj
 0001:00004640       SL_GetModemStatus          10005640 f   ser16950.obj
 0001:000046a4       SL_PurgeComm               100056a4 f   ser16950.obj
 0001:000047b4       SL_XmitComChar             100057b4 f   ser16950.obj
 0001:000048f4       SL_PowerOff                100058f4 f   ser16950.obj
 0001:00004c28       SL_PowerOn                 10005c28 f   ser16950.obj
 0001:00004f40       SL_SetDCB                  10005f40 f   ser16950.obj
 0001:000051ec       SL_SetCommTimeouts         100061ec f   ser16950.obj
 0001:00005208       SetFifoCtrlLevels          10006208 f   ser16950.obj
 0001:00005384       SetInternalLoopback        10006384 f   ser16950.obj
 0001:000053e4       SaveBaudrateMap            100063e4 f   ser16950.obj
 0001:000055f0       RegSetDeviceValue          100065f0 f   ser16950.obj
 0001:0000565c       SL_Ioctl                   1000665c f   ser16950.obj
 0001:00005904       SL_EnableXmit              10006904 f   ser16950.obj
 0001:00005960       SL_DisableXmit             10006960 f   ser16950.obj
 0001:000059bc       GetRegMultiDword           100069bc f   oxser.obj
 0001:00005a64       Ser_GetRegistryData        10006a64 f   oxser.obj
 0001:000062bc       Ser_Ioctl                  100072bc f   oxser.obj
 0001:00006440       GetSerialObject            10007440 f   oxser.obj
 0001:00006480       DisableThreadLibraryCalls  10007480 f   coredll:COREDLL.dll
 0001:00006490       LeaveCriticalSection       10007490 f   coredll:COREDLL.dll
 0001:000064a0       EventModify                100074a0 f   coredll:COREDLL.dll
 0001:000064b0       SetProcPermissions         100074b0 f   coredll:COREDLL.dll
 0001:000064c0       EnterCriticalSection       100074c0 f   coredll:COREDLL.dll
 0001:000064d0       InterlockedDecrement       100074d0 f   coredll:COREDLL.dll
 0001:000064e0       InterlockedIncrement       100074e0 f   coredll:COREDLL.dll
 0001:000064f0       ExitThread                 100074f0 f   coredll:COREDLL.dll
 0001:00006500       CreateThread               10007500 f   coredll:COREDLL.dll
 0001:00006510       InterruptDone              10007510 f   coredll:COREDLL.dll
 0001:00006520       InterruptInitialize        10007520 f   coredll:COREDLL.dll
 0001:00006530       WaitForSingleObject        10007530 f   coredll:COREDLL.dll
 0001:00006540       Sleep                      10007540 f   coredll:COREDLL.dll
 0001:00006550       InterruptDisable           10007550 f   coredll:COREDLL.dll
 0001:00006560       CloseHandle                10007560 f   coredll:COREDLL.dll
 0001:00006570       CeSetThreadPriority        10007570 f   coredll:COREDLL.dll
 0001:00006580       CeGetThreadPriority        10007580 f   coredll:COREDLL.dll
 0001:00006590       memcpy                     10007590 f   coredll:COREDLL.dll
 0001:000065a0       LocalFree                  100075a0 f   coredll:COREDLL.dll
 0001:000065b0       RegCloseKey                100075b0 f   coredll:COREDLL.dll
 0001:000065c0       RegQueryValueExW           100075c0 f   coredll:COREDLL.dll
 0001:000065d0       OpenDeviceKey              100075d0 f   coredll:COREDLL.dll
 0001:000065e0       CreateEventW               100075e0 f   coredll:COREDLL.dll
 0001:000065f0       InitializeCriticalSection  100075f0 f   coredll:COREDLL.dll
 0001:00006600       LocalAlloc                 10007600 f   coredll:COREDLL.dll
 0001:00006610       DeleteCriticalSection      10007610 f   coredll:COREDLL.dll
 0001:00006620       SetLastError               10007620 f   coredll:COREDLL.dll
 0001:00006630       memset                     10007630 f   coredll:COREDLL.dll
 0001:00006640       SetThreadPriority          10007640 f   coredll:COREDLL.dll
 0001:00006650       GetTickCount               10007650 f   coredll:COREDLL.dll
 0001:00006660       GetCurrentPermissions      10007660 f   coredll:COREDLL.dll
 0001:00006670       InterlockedExchange        10007670 f   coredll:COREDLL.dll
 0001:00006680       __C_specific_handler       10007680 f   coredll:COREDLL.dll
 0001:00006690       FreePhysMem                10007690 f   coredll:COREDLL.dll
 0001:000066a0       LoadIntChainHandler        100076a0 f   coredll:COREDLL.dll
 0001:000066b0       KernelLibIoControl         100076b0 f   coredll:COREDLL.dll
 0001:000066c0       _ultow                     100076c0 f   coredll:COREDLL.dll
 0001:000066d0       wcslen                     100076d0 f   coredll:COREDLL.dll
 0001:000066e0       RegSetValueExW             100076e0 f   coredll:COREDLL.dll
 0001:000066f0       wcstoul                    100076f0 f   coredll:COREDLL.dll
 0001:00006700       DDKReg_GetWindowInfo       10007700 f   coredll:COREDLL.dll
 0001:00006710       DDKReg_GetIsrInfo          10007710 f   coredll:COREDLL.dll
 0001:00006720       wcscpy                     10007720 f   coredll:COREDLL.dll
 0001:00006730       VirtualFree                10007730 f   coredll:COREDLL.dll
 0001:00006740       READ_PORT_UCHAR            10007740 f   ceddk:CEDDK.dll
 0001:00006750       READ_REGISTER_UCHAR        10007750 f   ceddk:CEDDK.dll
 0001:00006760       WRITE_PORT_UCHAR           10007760 f   ceddk:CEDDK.dll
 0001:00006770       WRITE_REGISTER_UCHAR       10007770 f   ceddk:CEDDK.dll
 0001:00006780       TransBusAddrToStatic       10007780 f   ceddk:CEDDK.dll
 0001:00006790       TransBusAddrToVirtual      10007790 f   ceddk:CEDDK.dll
 0001:000067a0       MmUnmapIoSpace             100077a0 f   ceddk:CEDDK.dll
 0001:000067b0       _DllMainCRTStartup         100077b0 f   corelibc:pegdmain.obj
 0001:00006848       _cinit                     10007848 f   corelibc:crt0dat.obj
 0001:00006988       _cexit                     10007988 f   corelibc:crt0dat.obj
 0001:000069a4       DllMain                    100079a4 f   corelibc:dllmain.obj
 0001:00006c00       __IMPORT_DESCRIPTOR_COREDLL 10007c00     coredll:COREDLL.dll
 0001:00006c14       __IMPORT_DESCRIPTOR_CEDDK  10007c14     ceddk:CEDDK.dll
 0001:00006c28       __NULL_IMPORT_DESCRIPTOR   10007c28     coredll:COREDLL.dll
 0002:00000000       __imp_TransBusAddrToVirtual 10008000     ceddk:CEDDK.dll
 0002:00000004       __imp_TransBusAddrToStatic 10008004     ceddk:CEDDK.dll
 0002:00000008       __imp_WRITE_REGISTER_UCHAR 10008008     ceddk:CEDDK.dll
 0002:0000000c       __imp_WRITE_PORT_UCHAR     1000800c     ceddk:CEDDK.dll
 0002:00000010       __imp_READ_REGISTER_UCHAR  10008010     ceddk:CEDDK.dll
 0002:00000014       __imp_READ_PORT_UCHAR      10008014     ceddk:CEDDK.dll
 0002:00000018       __imp_MmUnmapIoSpace       10008018     ceddk:CEDDK.dll
 0002:0000001c       \177CEDDK_NULL_THUNK_DATA  1000801c     ceddk:CEDDK.dll
 0002:00000020       __imp_CreateThread         10008020     coredll:COREDLL.dll
 0002:00000024       __imp_InterruptDone        10008024     coredll:COREDLL.dll
 0002:00000028       __imp_InterruptInitialize  10008028     coredll:COREDLL.dll
 0002:0000002c       __imp_WaitForSingleObject  1000802c     coredll:COREDLL.dll
 0002:00000030       __imp_Sleep                10008030     coredll:COREDLL.dll
 0002:00000034       __imp_InterruptDisable     10008034     coredll:COREDLL.dll
 0002:00000038       __imp_CloseHandle          10008038     coredll:COREDLL.dll
 0002:0000003c       __imp_CeSetThreadPriority  1000803c     coredll:COREDLL.dll
 0002:00000040       __imp_CeGetThreadPriority  10008040     coredll:COREDLL.dll
 0002:00000044       __imp_memcpy               10008044     coredll:COREDLL.dll
 0002:00000048       __imp_LocalFree            10008048     coredll:COREDLL.dll
 0002:0000004c       __imp_RegCloseKey          1000804c     coredll:COREDLL.dll
 0002:00000050       __imp_RegQueryValueExW     10008050     coredll:COREDLL.dll
 0002:00000054       __imp_OpenDeviceKey        10008054     coredll:COREDLL.dll
 0002:00000058       __imp_CreateEventW         10008058     coredll:COREDLL.dll
 0002:0000005c       __imp_InitializeCriticalSection 1000805c     coredll:COREDLL.dll
 0002:00000060       __imp_LocalAlloc           10008060     coredll:COREDLL.dll
 0002:00000064       __imp_DeleteCriticalSection 10008064     coredll:COREDLL.dll
 0002:00000068       __imp_SetLastError         10008068     coredll:COREDLL.dll
 0002:0000006c       __imp_ExitThread           1000806c     coredll:COREDLL.dll
 0002:00000070       __imp_SetThreadPriority    10008070     coredll:COREDLL.dll
 0002:00000074       __imp_GetTickCount         10008074     coredll:COREDLL.dll
 0002:00000078       __imp_GetCurrentPermissions 10008078     coredll:COREDLL.dll
 0002:0000007c       __imp_InterlockedExchange  1000807c     coredll:COREDLL.dll
 0002:00000080       __imp___rt_sdiv            10008080     coredll:COREDLL.dll
 0002:00000084       __imp___C_specific_handler 10008084     coredll:COREDLL.dll
 0002:00000088       __imp_FreePhysMem          10008088     coredll:COREDLL.dll
 0002:0000008c       __imp_LoadIntChainHandler  1000808c     coredll:COREDLL.dll
 0002:00000090       __imp_KernelLibIoControl   10008090     coredll:COREDLL.dll
 0002:00000094       __imp__ultow               10008094     coredll:COREDLL.dll
 0002:00000098       __imp_wcslen               10008098     coredll:COREDLL.dll
 0002:0000009c       __imp_RegSetValueExW       1000809c     coredll:COREDLL.dll
 0002:000000a0       __imp_wcstoul              100080a0     coredll:COREDLL.dll
 0002:000000a4       __imp_DDKReg_GetWindowInfo 100080a4     coredll:COREDLL.dll
 0002:000000a8       __imp_DDKReg_GetIsrInfo    100080a8     coredll:COREDLL.dll
 0002:000000ac       __imp_wcscpy               100080ac     coredll:COREDLL.dll
 0002:000000b0       __imp_VirtualFree          100080b0     coredll:COREDLL.dll
 0002:000000b4       __imp_InterlockedIncrement 100080b4     coredll:COREDLL.dll
 0002:000000b8       __imp_InterlockedDecrement 100080b8     coredll:COREDLL.dll
 0002:000000bc       __imp_EnterCriticalSection 100080bc     coredll:COREDLL.dll
 0002:000000c0       __imp_SetProcPermissions   100080c0     coredll:COREDLL.dll
 0002:000000c4       __imp_EventModify          100080c4     coredll:COREDLL.dll
 0002:000000c8       __imp_LeaveCriticalSection 100080c8     coredll:COREDLL.dll
 0002:000000cc       __imp_memset               100080cc     coredll:COREDLL.dll
 0002:000000d0       __imp_DisableThreadLibraryCalls 100080d0     coredll:COREDLL.dll
 0002:000000d4       \177COREDLL_NULL_THUNK_DATA 100080d4     coredll:COREDLL.dll
 0002:000000d8       __xc_a                     100080d8     corelibc:crt0init.obj
 0002:000000dc       __xc_z                     100080dc     corelibc:crt0init.obj
 0002:000000e0       __xi_a                     100080e0     corelibc:crt0init.obj
 0002:000000e4       __xi_z                     100080e4     corelibc:crt0init.obj
 0002:000000e8       __xp_a                     100080e8     corelibc:crt0init.obj
 0002:000000ec       __xp_z                     100080ec     corelibc:crt0init.obj
 0002:000000f0       __xt_a                     100080f0     corelibc:crt0init.obj
 0002:000000f4       __xt_z                     100080f4     corelibc:crt0init.obj
 0002:00000100       _exitflag                  10008100     <common>
 0002:00000104       __onexitend                10008104     <common>
 0002:00000108       __onexitbegin              10008108     <common>
 0002:0000010c       _pRawDllMain               1000810c     <common>

 entry point at        0001:000067b0

 Static symbols

 0001:00000718       SerialDispatchThread       10001718 f   mdd.obj
 0001:00005e20       SerInit                    10006e20 f   oxser.obj
 0001:00005fb8       Ser_InternalMapRegisterAddresses 10006fb8 f   oxser.obj
 0001:0000607c       SerSetOutputMode           1000707c f   oxser.obj
 0001:00006080       SerClose                   10007080 f   oxser.obj
 0001:00006130       SerDeinit                  10007130 f   oxser.obj
 0001:0000619c       SerGetCommProperties       1000719c f   oxser.obj
 0001:000061c0       SerPowerOff                100071c0 f   oxser.obj
 0001:000061e8       SerPowerOn                 100071e8 f   oxser.obj
 0001:00006220       SerEnableIR                10007220 f   oxser.obj
 0001:00006244       SerDisableIR               10007244 f   oxser.obj
 0001:00006268       SerOpen                    10007268 f   oxser.obj
 0001:0000687c       _initterm                  1000787c f   corelibc:crt0dat.obj
 0001:000068b0       doexit                     100078b0 f   corelibc:crt0dat.obj
